:100000000C9417060C94CA280C94F7280C943F06FD
:100010000C943F060C943F060C943F060C943F064C
:100020000C943F060C943F060C94020C0C943F0673
:100030000C943F060C943F060C943F060C943F062C
:100040000C9424290C943F060C94BC2C0C94F72C93
:100050000C943F060C943F060C943F060C943F060C
:100060000C943F060C943F06181C1F1C1F1C181CE8
:100070001F1C1F1C1F1C1F1C1F1C1F1C1F1C1F1CA8
:100080001F1C1F1C1F1C1F1C1F1C8D1B1F1C1F1C2B
:100090001F1C1F1C1F1CF01A1F1C1F1C1F1C1F1CB9
:1000A0001F1C1F1C1F1C1F1C1F1C1F1C1F1C1F1C78
:1000B0001F1C1F1C1F1C991B991B991B991B991B0B
:1000C000991B991B991B991B1F1C1F1C1F1C1F1C74
:1000D0001F1C1F1CF51A981B981B981B981B1F1C94
:1000E000A91BB11BB91BC11BC91BD11BD91BE11B10
:1000F000EB1BF51BFF1B091C3C1BFC1A1F1C1F1CC8
:100100001F1C1F1C8D1B1F1C1F1C1F1C1F1C1F1CAA
:100110001F1C1F1C1F1C971B971B971B971B1F1C2B
:10012000A91BB11BB91BC11BC91BD11BD91BE11BCF
:10013000EB1BF51BFF1B091C3C1BFC1A1F1C1F1C87
:100140001F1C1F1C8D1B501C501C501C501C501C75
:10015000501C501C501C501C501C501C501C501C3F
:10016000701D701D701D701D701D701D971CA11CD1
:10017000AB1CB51C1B1D251D331D441DE11D511E4F
:10018000221E271E2C1E311E361E3B1E401E511ED7
:100190004B1E5E2573257F2588259525BB25C32508
:1001A000E625D325456E746572206D656E752E2E1D
:1001B0002E00546F67676C6564206D6963726F50C1
:1001C000504D00546F67676C656420696E76657288
:1001D0007465642050504D2100546F67676C6564EE
:1001E000205458206D7574696E672100546F6767DD
:1001F0006C65642074656C656D657472792100505E
:10020000726F746F636F6C206572726F72207769A2
:1002100074682052580054696D656F757420776852
:10022000656E20636F6E6E656374696E6720746FB0
:1002300020525800507265737320616E79206B658F
:100240007920746F2063616E63656C00436F6E6E1E
:10025000656374696E6720746F2052582C20706F2C
:100260007765722075702074686520525820287751
:100270006974682062696E6420706C7567206966B5
:10028000206E6F74207573696E6720616C77617979
:10029000732062696E642900546F67676C6564201F
:1002A00027696D6D656469617465206F757470751B
:1002B000742700546F67676C65642027736C6176E0
:1002C00065206D6F64652700546F67676C656420F7
:1002D00027616C776179732062696E642700546FBF
:1002E00067676C65642050504D206368616E6E6571
:1002F0006C206C696D6974005365742052535349C6
:1003000020696E6A656374696F6E206368616E6EE2
:10031000656C2028303D3D64697361626C6529001D
:100320005365742050504D206D696E696D756D2058
:1003300073796E630053657420626561636F6E202C
:10034000696E74657276616C0053657420626561D4
:10035000636F6E2064656C6179005365742062651B
:1003600061636F6E206672657175656E6379206971
:100370006E20487A3A20303D64697361626C652C66
:100380002050783D504D52206368616E6E656C2040
:10039000782C2046783D465253206368616E6E6526
:1003A0006C2078005365742050574D2073746F7023
:1003B0002064656C61792028302064697361626C07
:1003C00065642C20312D323535203D3D20302E31D5
:1003D00073202D2035306D696E29005365742050CF
:1003E000504D2073746F702064656C6179202830E3
:1003F0002064697361626C65642C20312D3235355F
:10040000203D3D20302E3173202D2035306D696E1A
:100410002900536574206661696C736166652064A8
:10042000656C61792028302064697361626C656451
:100430002C20312D323535203D3D20302E3173209A
:100440002D2035306D696E29002A2A2A2A2A2A2A67
:100450002A2A2A2A2A2A2A2A2A2A2A2A2A2A2A2AFC
:100460002A2A2A2A2A2A0052582041636B656420CE
:100470002D2072657665727420737563636573737E
:1004800066756C21002A2A2A2A2A2A2A2A2A2A2A36
:100490002A2A2A2A2A2A2A2A2A2A2A2A2A2A2A2ABC
:1004A0002A2A002A2A2A2A2A2A2A2A2A2A2A2A2AD6
:1004B0002A2A2A2A2A2A2A2A2A2A2A2A2A2A2A2A9C
:1004C0000052582041636B6564202D207570646173
:1004D0007465207375636365737366756C21002A98
:1004E0002A2A2A2A2A2A2A2A2A2A2A2A2A2A2A2A6C
:1004F0002A2A2A2A2A2A2A2A2A2A2A2A0056616CE1
:1005000069642063686F69636573206172653A206E
:100510005B315D2D5B31365D20286368616E6E65F1
:100520006C20312D31362900536574206F7574703D
:10053000757420666F7220706F727420005B585D56
:100540002061626F7274206368616E6765732061F9
:100550006E64206578697420525820636F6E6669F6
:1005600067005B535D207361766520736574746901
:100570006E677320746F205258005B525D20726565
:10058000766572742052582073657474696E67734F
:1005900020746F2064656661756C747300557365B3
:1005A000206E756D62657273205B312D445D207421
:1005B0006F206564697420706F727473205B452DC1
:1005C000515D20666F722073657474696E67730085
:1005D000202D20726563656976657220636F6E6693
:1005E0006967757261746F722C207278207377203E
:1005F000000A0A6F70656E4C52536E672000536597
:10060000742073657269616C2062617564726174D3
:10061000653A200056616C69642063686F696365A0
:10062000733A2031202D20342B34202F2032202DDE
:100630002038202F2033202D20382B34202F203419
:10064000202D203132202F2035202D2031322B3407
:10065000202F2036202D203136005365742043682A
:10066000616E6E656C20636F6E6669673A20005339
:1006700065742044617461726174652028302D3284
:10068000293A200053657420486F70206368616EBA
:100690006E656C7320286D61782032342C20736570
:1006A0007061726174656420627920636F6D6D6141
:1006B00073292076616C69642076616C756573209E
:1006C000312D3235353A2000536574206368616EF0
:1006D0006E656C2073706163696E672028783130B5
:1006E0006B487A293A200053657420524620706F77
:1006F0007765722028302D37293A20005365742001
:100700005246206D616769632028686578292065F5
:100710002E672E20307844454144463030443A20FC
:10072000005365742062617365206672657175653A
:100730006E63792028696E20487A293A20005B5A36
:100740005D20656E74657220726563656976657299
:1007500020636F6E66696775726174696F6E20756C
:1007600074696C79005B465D20646973706C6179B3
:100770002061637475616C206672657175656E6366
:100780006965732075736564005B525D2063616CFD
:1007900063756C6174652072616E646F6D206B654A
:1007A0007920616E6420686F70206C697374005BDF
:1007B000495D207265696E697469616C697A65204A
:1007C00073657474696E677320746F20736B6574DE
:1007D00063682064656661756C7473005B585D20A6
:1007E000726576657274206368616E6765732061F7
:1007F0006E642065786974206D656E75005B535D6D
:1008000020736176652073657474696E67732074F4
:100810006F20454550524F4D20616E6420657869C8
:1008200074206D656E7500557365206E756D62651B
:100830007273205B302D395D20746F20656469749C
:1008400020706172616D657465727300202D205394
:10085000797374656D20636F6E6669677572617414
:10086000696F6E000A0A6F70656E4C52536E672096
:10087000005129204F7574707574206265666F721F
:1008800065206C696E6B20283D465329203A200074
:10089000502920536C617665206D6F646520286552
:1008A00078706572696D656E74616C293A20004FCD
:1008B000292054696D65642042494E4420617420AA
:1008C0007374617274757020203A20004E29205094
:1008D000504D206F7574707574206C696D69746506
:1008E0006420202020203A200044495341424C45B6
:1008F00044004D292050504D205253534920746FCD
:10090000206368616E6E656C202020203A20004CC8
:10091000292050504D206D696E696D756D20737979
:100920006E63202875732920203A200044495341E2
:10093000424C4544004B29204661696C73616665F1
:1009400020626561636F6E20696E74762E20283197
:100950002D32353573293A20004A29204661696CC9
:100960007361666520626561636F6E2064656C61AA
:10097000792028302D323535203D3E20313073200E
:100980002D203135306D696E293A200049292046E5
:1009900061696C7361666520626561636F6E206674
:1009A00072712E203A200048292050574D20737430
:1009B0006F702064656C6179202020202020203A0F
:1009C000200047292050504D2073746F70206465BB
:1009D0006C6179202020202020203A200046292008
:1009E0004661696C736166652064656C617920207D
:1009F00020202020203A200050574D206368616E4F
:100A00006E656C200066756E6374696F6E3A2000C7
:100A10002920706F72742000506F776572546F7761
:100A2000657200445446205548462033322D626991
:100A3000742031306368004F70656E4C52536E679E
:100A40005258206D696E6920342F36636800466CF9
:100A50007974726F6E2F4F72616E676552582055B0
:100A600048462038636800525820747970653A20EF
:100A70000044697361626C656400487A00203D3D02
:100A8000200043616C63756C617465642070616300
:100A90006B657420696E74657276616C3A200042F1
:100AA00029204D6963726F202868616C6629205087
:100AB000504D202020203A00412920496E76657251
:100AC0007465642050504D20696E20202020203A0B
:100AD000003029204D7574652062757A7A65722020
:100AE000286D6F73746C79293A0039292053657227
:100AF00069616C2062617564726174653A00736D3E
:100B0000617274506F7274004672536B7900547244
:100B1000616E73706172656E740044697361626CBA
:100B200065640038292054656C656D657472793A86
:100B300020202020202020003729204368616E6E6D
:100B4000656C20636F6E6669673A20200036292045
:100B500044617461726174652028302D32293A2015
:100B6000202000352920486F70206368616E6E6513
:100B70006C733A2020202020003429204368616EC5
:100B80006E656C2073706163696E673A2020003374
:100B90002920524620706F7765722028302D372922
:100BA0003A202020003229205246206D6167696377
:100BB0003A202020202020202020003129204261BE
:100BC0007365206672657175656E63793A202020C1
:100BD0000000000000240027002A0000000000257B
:100BE0000028002B0000000000230026002900043C
:100BF00004040404040404020202020202030303C4
:100C000003030301020408102040800102040810BD
:100C1000200102040810200000000700020100006B
:100C20000304060000000000000000009F2E1124B5
:100C30001FBECFEFD8E0DEBFCDBF13E0A0E0B1E034
:100C4000E0E8FFE502C005900D92A639B107D9F79B
:100C500016E0A6E9B3E001C01D92A934B107E1F79F
:100C60001CE0CEE2DCE004C02297FE010E949B2F34
:100C7000CC32D107C9F70E94E42E0C94BE2F0C94FD
:100C80000000A0E0B0E0E7E4F6E00C946A2FEC018D
:100C9000A880B980CA80DB80A114B104C104D1044A
:100CA00041F484E2A82E89EDB82E8BE5C82E87E0AA
:100CB000D82EC601B5012DE133EF41E050E00E948E
:100CC000472F27EA31E440E050E00E94F32E7B01F9
:100CD0008C01C601B5012DE133EF41E050E00E94E7
:100CE000472FCA01B9012CEE34EF4FEF5FEF0E949E
:100CF000F32E6E0D7F1D801F911F97FF04C0615062
:100D0000704080409048688379838A839B839B01ED
:100D1000AC015F77B901CA01CDB7DEB7EAE00C9448
:100D2000862F0E944106089581EB92E00E944106C1
:100D300008956093B1027093B2028093B3029093CE
:100D4000B4020895A0E0B0E0E8EAF6E00C94632F66
:100D5000EC012B016A016115710519F0FB0191830A
:100D60008083C114D10449F0C6010297839728F00B
:100D700020E030E040E050E0DCC0A9908A2D90E017
:100D80000E94B32F892BC9F7FDE2AF1621F4A99079
:100D90003324339405C08BE2A81609F4A9903324B8
:100DA000C114D10421F0E0E1CE16D10411F5F0E335
:100DB000AF1669F48881883711F0883541F4A9802D
:100DC000229682E0382A20E1C22ED12C12C0C11412
:100DD000D10479F4E0E3AE1659F199E9E92E99E9E5
:100DE000F92E99E9092F99E1192F8AE0C82ED12C03
:100DF0003AC0FAE0CF16D10491F080E1C816D104D0
:100E000029F0E8E0CE16D104F9F415C0BFEFEB2EBF
:100E1000BFEFFB2EBFEF0B2FBFE01B2F24C0A9E9B4
:100E2000EA2EA9E9FA2EA9E90A2FA9E11A2F1BC077
:100E3000F8E0CF2ED12CEFEFEE2EEFEFFE2EEFEFFE
:100E40000E2FEFE11E2F0FC09601442737FD40956E
:100E5000542F6FEF7FEF8FEF9FEF0E94252FC90177
:100E6000DA017C018D0120E030E040E050E060E0FC
:100E70003601882477FC8094982C70EDB72EBA0C3C
:100E8000F9E0FB1570F48A2D81548A3118F499EC3D
:100E9000B92E06C08A2D81568A3148F589EAB82EC6
:100EA000BA0C8B2D90E08C159D050CF56F3FE9F089
:100EB000E216F30604071507B8F0CA01B901A40148
:100EC00093010E94F32E9B01AC018B2D90E0A0E0DA
:100ED000B0E0280F391F4A1F5B1F281739074A0740
:100EE0005B0710F061E001C06FEFA990C6CF41141D
:100EF000510451F0662311F0219703C031FE04C064
:100F00002297F201D183C08330FE07C050954095EF
:100F1000309521953F4F4F4F5F4F67FF0AC082E2E8
:100F200090E090934806809347062FEF3FEF4FEFF6
:100F30005FEFB901CA01CDB7DEB7E1E10C947F2FB5
:100F4000FC0188279927E89421912032E9F3293080
:100F500010F02E30C8F32B3241F02D3239F4689462
:100F600004C00E94F507820F911D219120532A3061
:100F7000C0F31EF4909581959F4F089546E953E084
:100F80000E94C3070895009731F4DA018D919C9176
:100F9000009709F40EC0DC01FB013D912191222351
:100FA00019F03217C9F3FACF332331F4DA011D9265
:100FB0001C928827992708951197AF93BF93FB013F
:100FC0003D912191321771F4332321F48827992719
:100FD000119702C01E921196FA01A193B0839F91BE
:100FE0008F910895222369F7EACF7AE0979F902D99
:100FF000879F802D910D1124089580919803813051
:1010000019F482E08093980380919803833019F457
:1010100084E0809398030895009721F19C0140E0BB
:1010200050E068E478EE81E090E00E94472FC9012B
:10103000DA018F3F9105A105B10531F028F08FEF5E
:1010400090E0A0E0B0E008C00097A105B10521F450
:1010500081E090E0A0E0B0E08093B3008091B00028
:10106000806103C08091B0008F7E8093B0000895AE
:10107000E3E0F0E089E080935700849190E086708F
:10108000863009F491E0892F08951F93182F0E944C
:101090003808882379F09FB781E080938F05F89412
:1010A000A89588E18093600010936000112309F0F7
:1010B000A8959FBF1F910895382F20E080912105AA
:1010C000909122058227932740E061E270E19C0124
:1010D000220F331F97FF04C0C9018627972701C03D
:1010E000C9014F5F483099F79093220580932105FD
:1010F000089586E38093BE0380E092ECA1E0B0E027
:101100008093BF039093C003A093C103B093C20325
:1011100087E08093CB0380EC92E9ADEEB9E1809358
:10112000C3039093C403A093C503B093C60385E0A3
:101130008093CC038DEE9EEFADEABEED8093C703A6
:101140009093C803A093C903B093CA03ADECB3E076
:1011500080E090E0863010F0E0E004C0FC01E05850
:10116000FC4FE081ED9301968831910599F782E07B
:101170008093E5038AE08093E603089580EC91ED87
:10118000A8E9BBE180939B0390939C03A0939D03EC
:10119000B0939E0310929F031092A0031092A1039C
:1011A0001092A20308958436910520F4BC0180E0DA
:1011B00090E025C08E3B910550F48A559040BC01CB
:1011C00080E090E02AE030E040E050E016C0823D50
:1011D000910550F4845B9040BC0180E090E024E6EF
:1011E00030E040E050E009C08D5C9040BC0180E000
:1011F00090E028E532E040E050E00E94F32E24E643
:1012000030E040E050E00E94F32E089590E08C59C9
:101210009F4F0E94D3080895DC019896EC91F0E06E
:10122000E770F070E858FC4F808108958F929F928C
:10123000AF92BF92CF92DF92EF92FF920F931F93E4
:101240008C010E940C09D80197962C9130E043E163
:1012500050E0249FF001259FF00D349FF00D1124E4
:10126000EB54FD4F80809180A280B38090E00F9678
:10127000AA2797FDA095BA2FBC01CD0120E43FE13C
:101280004DE750E00E94F32EA50194010E94252F06
:1012900069017A0180ED97E0A0E0B0E0C80ED91EA8
:1012A000EA1EFB1ED80198968C91887181F060E04F
:1012B0007EEE8AEB9BE0A50194010E94252F285128
:1012C0003C4F4F4F5F4FC20ED31EE41EF51E87EEFC
:1012D00093E0A0E0B0E0C80ED91EEA1EFB1EC701D5
:1012E000B60128EE33E040E050E00E94252FCA010D
:1012F000B90128EE33E040E050E00E94F32E1F9148
:101300000F91FF90EF90DF90CF90BF90AF909F90A4
:101310008F9008958F3F910509F010F480E00895B3
:1013200022E08030920710F481E0089580509340CD
:1013300010F083E0089582E00895CF92DF92FF924B
:101340000F931F93CF93DF93F82FEB016A01182FB0
:101350001695E0E088819981D6018C938A819B81E2
:1013600011968C9311978C819D8112968C93129774
:101370008E819F8113968C931397288139814A819E
:101380005B816C817D818E819F819295990F990FF0
:10139000907C832F8370982B852F8370880F880F04
:1013A000982B872F83708295807F982B14969C931F
:1013B00085E090E0C80ED91E2896EF5F1E1750F604
:1013C000F0FF21C0888199810E948A09F82E8A81C4
:1013D0009B810E948A09182F8C819D810E948A0915
:1013E000082F8E819F810E948A09F294FF0CFF0CC6
:1013F00070ECF7221295107F1F29182B000F000F99
:10140000012BD6010C93DF91CF911F910F91FF908B
:10141000DF90CF90089523E08032920718F420E007
:1014200030E026C023E0883E920748F49C012F510B
:10143000334054E0369527955A95E1F719C027E0D7
:10144000803D920720F49C012C5D334011C028E0C0
:101450008839920718F02FEF33E00AC09C01285C0E
:10146000374044E0369527954A95E1F72D503C4F9B
:10147000C90108958C30910548F49C0174E0220F55
:10148000331F7A95E1F7285D3C4F17C023E0843F76
:10149000920720F49C0124523C4F0FC024E080307E
:1014A000920718F020E938E008C09C012657334F16
:1014B00064E0220F331F6A95E1F7C90108959C018A
:1014C0003695279525753575821B930B9C013695AE
:1014D0002795369527952373337383739373280F5A
:1014E000391FC901E4E096958795EA95E1F7820FE7
:1014F000931F8F709F7021E031E0AC01429FC001CB
:10150000439F900D529F900D1124892F0895882399
:1015100039F02D9800002B9A00002D9A00000895B4
:101520002D9800002B9800002D9A000008952D9A08
:10153000000083B12D98000090E0B4E09695879567
:10154000BA95E1F7817008950F931F93082F5C9A65
:101550002D985C9810E0802F80780E94870A000FF9
:101560001F5F1830C1F72D981F910F9108958F7745
:101570000E94A40A08950F931F93082F10E0802F54
:1015800080780E94870A000F1F5F1830C1F72D98DE
:101590001F910F9108950F931F932D9880E000E005
:1015A000182F110F0E94970A810F0F5F0830C1F7A3
:1015B0001F910F9108950E94B70A0E94CB0A5C9A6E
:1015C00008951F93162F80680E94A40A812F0E94FD
:1015D000BB0A5C9A1F9108951F931091C7031827A7
:1015E000EEEBF3E0E80FF11D89E767850E94E10A61
:1015F0008DE3612F0E94E10A82E4612F0E94E10ADB
:101600001F91089586E20E94DB0A08950F931F93AD
:101610008C018CE1F80164810E94E10A8DE1F801FE
:1016200065810E94E10A8EE1F80166810E94E10A6B
:1016300080E2F80167810E94E10A81E2F801608599
:101640000E94E10A82E2F80161850E94E10A83E2D8
:10165000F80162850E94E10A84E2F80163850E9434
:10166000E10A85E2F80164850E94E10A8AE2F80154
:1016700065850E94E10A8EE6F80166850E94E10A0E
:101680008FE6F80167850E94E10A80E7F80160892A
:101690000E94E10A81E7F80161890E94E10A82E77C
:1016A000F80162890E94E10A1F910F910895EF925B
:1016B000FF920F931F93CF93DF937B018C016030D8
:1016C00028E372072CE982072CE1920728F520E82D
:1016D00036E948E950E00E94252FE9016897B901F1
:1016E00080E090E020E839E647E65FEF0E94F32EC5
:1016F0006E0D7F1D801F911F32E0660F771F881FC0
:10170000991F3A95D1F721E732E040E050E00E947E
:10171000252F890180E421C020E03DE241E351E032
:101720000E94252FE9016897B90180E090E020E050
:1017300033ED4EEC5EEF0E94F32E6E0D7F1D801F89
:10174000911F660F771F881F991F21E732E040E045
:1017500050E00E94252F890180E69E012F71622FA3
:10176000680F85E70E94E10A86E7612F0E94E10A7F
:1017700087E7602F0E94E10ACDB7DEB7E6E00C9460
:101780008A2F87E061E00E94E10A8EE764E20E940E
:10179000E10A88E063E00E94E10A88E060E00E94DC
:1017A000E10A87E065E00E94E10A85E062E00E94CC
:1017B000E10A83E00E94DB0A8093E70384E00E9451
:1017C000DB0A8093E8030895582F40918C04842FFE
:1017D00090E0FC01EF70F0709F012F5F3F4F64E0DD
:1017E000959587956A95E1F72817390751F0E458E0
:1017F000FB4F5083842F8F5F8F70407F842B8093AB
:101800008C0408951F920F920FB60F9211241F930C
:101810002F933F934F935F936F937F938F939F93F8
:10182000AF93BF93CF93DF93EF93FF93C091860065
:10183000D09187002091CE043091CF048091AD04E7
:10184000882309F047C0CE01821B930B9C01809135
:101850009F0385FD02C03695279599E0253C390701
:1018600008F1809147038630D0F0809147038F3F85
:10187000B1F020E00EC0E22FF0E0EE0FFF1FDF011D
:10188000A255BB4F8D919C91E95DFC4F9183808364
:101890002F5F80914703281770F31092AC041092C9
:1018A000470318C082E02D3B380760F18091470361
:1018B000803140F510914703C9010E940B0AE12FC6
:1018C000F0E0EE0FFF1FE255FB4F918380831F5F17
:1018D00010934703D093CF04C093CE04FF91EF91B0
:1018E000DF91CF91BF91AF919F918F917F916F9138
:1018F0005F914F913F912F911F910F900FBE0F90CD
:101900001F9018958FEF80934703E4CF83E0809377
:1019100080008AE98093810080919F0386FD05C045
:10192000809181008064809381008FEF9FEF90937E
:1019300089008093880080916F00806280936F009F
:1019400008956F3020F086958695805408958DE037
:10195000689F802D11240895882319F460E071E0B8
:1019600002C063E071E085E296E00E94A72C089532
:10197000A0E0B0E0EEEBFCE00C946C2F182F0E947E
:101980007A299B01AC0180911B0590911C05A091C7
:101990001D05B0911E0569017A01C81AD90AEA0A23
:1019A000FB0AD701C60189589341A040B04010F00E
:1019B00010921A0520931B0530931C0540931D05BA
:1019C00050931E052091AD04822F81508230E8F59E
:1019D00080911A05882309F44FC1813011F482E007
:1019E000BCC1803108F035C1E82FF0E0E255FB4F73
:1019F00010838F5F80931A05803109F0B0C1A0EB8E
:101A0000B4E0213039F41196EC911197E695E69502
:101A10008C9109C08D919C911197E92FE695E695DF
:101A2000E69596958795E03140F4F0E090E0EE0F72
:101A3000FF1FE95DFC4F918380831092AC041296E6
:101A400084E0AE3BB807E9F68AC1233009F004C14F
:101A500080911A05882321F41F3009F080C10CC140
:101A6000883130F4E82FF0E0E355FB4F108374C168
:101A7000883109F0EEC0112309F0EBC0C0E0D0E0DE
:101A80000BE010E0DE0163E0AA0FBB1F6A95E1F7EF
:101A9000C09FB001C19F700DD09F700D1124FB013C
:101AA000E255FB4F80812181922F97709595879504
:101AB000FD01EE0FFF1FE95DFC4F91838083FB0169
:101AC000E155FB4F30813695369536952181422F71
:101AD0004295440F407E842F832B2695269526958C
:101AE000922F977095958795FD01EE0FFF1FE75D8B
:101AF000FC4F91838083FB01E055FB4F80818295F1
:101B00008695869583704181942F990F990F292F7F
:101B1000282B429546954695437082818170880FA7
:101B2000880F382F342B35952795FD01EE0FFF1FB9
:101B3000E55DFC4F31832083FB01EE54FB4F308188
:101B400036952181422F479544274795842F832B33
:101B50002695922F977095958795FD01EE0FFF1FA3
:101B6000E35DFC4F91838083FB01ED54FB4F30819B
:101B700032953F702181422F4295407F842F832BE5
:101B800022952F70922F977095958795FD01EE0FF6
:101B9000FF1FE15DFC4F91838083FB01EC54FB4F01
:101BA0008081881F8827881F4181942F990F292FB2
:101BB000282B441F4427441F82818370880F382FAD
:101BC000342B35952795FD01EE0FFF1FEF5CFC4F81
:101BD00031832083FB01EA54FB4F308136953695E3
:101BE0002181422F4295440F440F407C842F832B48
:101BF00026952695922F977095958795AA0FBB1FCE
:101C0000FD01ED5CFC4F9183808369547B4FFB01A8
:101C100020812295269527704181342F330F330F71
:101C2000330F832F822B942F9295969597709595CD
:101C30008795AB5CBC4F11969C938E932196C230D6
:101C4000D10509F01FCF8091C40483FD02C010921A
:101C5000AC0410921A0583C0243009F080C0409172
:101C60001A05442359F4183AB1F41092220510923F
:101C7000210588EA0E945C0881E06FC0413019F4B8
:101C800010931F0504C0423031F410932005812FBA
:101C90000E945C085DC060912005262F30E0220F75
:101CA000331FE42FF0E0C90102968E179F0734F02E
:101CB000433268F7E555FB4F1083E9CF2D5F3F4F67
:101CC0004091210550912205E217F30749F4912F25
:101CD00080E048275927509322054093210538C0BA
:101CE000812F90E04817590789F580911F058130B1
:101CF00069F5613118F080E180932005D0902005CE
:101D00004EEAE42E44E0F42E00E010E01BC0F701A0
:101D1000D081C0E0818190E08C2B9D2B33E09695A3
:101D200087953A95E1F70E940B0AF801EE0FFF1F25
:101D3000E95DFC4F918380830F5F1F4F82E090E04D
:101D4000E80EF91E0D1518F31092AC0410921A0546
:101D500080911A05882319F08F5F80931A05CDB7FB
:101D6000DEB7E8E00C94882FFF920F931F93CF9378
:101D7000DF93182F092FF62E8EE30E94E10A212F00
:101D8000302FC901EC0110E005C08FE769910E9476
:101D9000E10A1F5F1F15C8F385E064E00E94E10AB5
:101DA00083E00E94DB0A8093E70384E00E94DB0A61
:101DB0008093E8030E947A296093E9037093EA0311
:101DC0008093EB039093EC0387E069E00E94E10AC3
:101DD00081E080939803CDB7DEB7E5E00C948B2FBC
:101DE0000E94B40E809198038130D9F40E947A2920
:101DF0002091E9033091EA034091EB035091EC0309
:101E0000621B730B840B950B605A7648814090409F
:101E100040F4E8CF85E296E067E071E00E94A72CED
:101E20000895809198038130A9F3089585E296E0A2
:101E30006EE70E945F2E0895A0E0B0E0E2E2FFE0CE
:101E40000C946B2F6C0185E296E06EE70E945F2E8A
:101E5000760100E010E0C0E0D0E0B0E2BB2E0AC0A6
:101E60000830110521F49E012095F6012087089481
:101E7000E11CF11CF7016081862F8D57823040F400
:101E800085E296E06DE70E945F2EF70160816B2589
:101E900085E296E00E945F2E0115110551F0F701D1
:101EA00080819E01280F311DC32FDD27C20FD31F54
:101EB000D0700F5F1F4F0930110591F6CDB7DEB717
:101EC000E9E00C94872FA9E0B0E0E9E6FFE00C948C
:101ED000722F382FE62F8091910490E0019664E2F2
:101EE00070E00E94122F982F8093910488E98983D3
:101EF00080E18A83913071F0913028F0923099F02E
:101F00009330E1F416C085E08B8381EF8C832F5FE3
:101F10002D8317C09B8381EF8C8384E6489FC0018B
:101F200011249D830EC084E08B8381EF8C833D83DD
:101F300008C09B8381EF8C83ED8303C00E94160F42
:101F400004C0CE0101960E941C0F2996E2E00C9479
:101F50008E2F0F931F93CF93DF93182F092F85E2B6
:101F600096E06EE70E945F2E212F302FC901EC0111
:101F700010E000E288818D57823040F485E296E0DF
:101F80006DE70E945F2E88818027888385E296E036
:101F900069910E945F2E1F5F193061F785E296E01C
:101FA0006EE70E945F2EDF91CF911F910F910895F0
:101FB000A9E0B0E0EEEDFFE00C94722F382F809195
:101FC0009104882379F48EEF89833A836B83842F7D
:101FD00090E0959587958C832D83198618861F82AE
:101FE0001E822FC040918C04842F90E09C012F70A2
:101FF000307054E0959587955A95E1F782179307CD
:1020000021F18DEF89831A821B82DE01149620E074
:1020100008C0E458FB4F80818D93405F2F5F2630CE
:1020200069F0842F90E0FC0134E0F595E7953A954E
:10203000E1F78F709070E817F90759F740938C0417
:102040002A83CE0101960E94A90F8091910490E00D
:10205000019666E070E00E94122F80939104299609
:10206000E2E00C948E2F9F92AF92BF92CF92DF92BC
:10207000EF92FF920F931F93B82EA62ED42EC22E4E
:10208000902E0E947A297B018C0180917B04209103
:102090008D0430918E0440918F04509190048823D8
:1020A000B1F0D801C701821B930BA40BB50B815E65
:1020B0009E42A040B04020F12C2DDC1408F42D2DC0
:1020C0008B2D6A2D422F292D0E94630F11C0D8013C
:1020D000C701821B930BA40BB50B81539547A040FE
:1020E000B04070F08B2D6A2D4D2D2C2D0E94D80FF5
:1020F000E0928D04F0928E0400938F04109390046C
:102100001F910F91FF90EF90DF90CF90BF90AF9015
:102110009F90089585E296E06091EE030E945F2E05
:1021200008951F93182F85E296E0612F0E945F2E7D
:102130008091EE0381278093EE031F9108951F93F2
:10214000192F0E949110812F0E9491101F910895C4
:10215000DF92EF92FF920F931F93D82E7B01109284
:10216000EE0305E216E0C80165EB0E945F2EC80190
:1021700062E60E945F2E8D2D0E949110C7010E9481
:102180009F101F910F91FF90EF90DF9008958CE0CA
:1021900060E00E94FF298BE061E00E94FF298DE052
:1021A00061E00E94FF2982E060E00E94FF2984E054
:1021B00061E00E94FF29089582E08093B00085E0ED
:1021C0008093B10083E061E00E94FF2983E060E03A
:1021D0000E946B2A08951F93182F0E947A296093FA
:1021E0008D0470938E0480938F04909390041093C9
:1021F0007B04112329F440E855E260E070E004C05C
:1022000040E051EE60E070E085E296E00E94652DCE
:102210001F91089583E00E94DB0A8093E70384E026
:102220000E94DB0A8093E80387E061E00E94E10AF4
:102230006AE070E080E090E00E94A0290E94C10B5B
:10224000000008959F92AF92BF92CF92DF920F93BA
:10225000DF93CF9300D000D0CDB7DEB7982E89E0C2
:1022600061E00E946B2A62E370E080E090E00E94EF
:10227000A02989E060E00E946B2A62E370E080E0C0
:1022800090E00E94A02983E00E94DB0A8093E7038C
:1022900084E00E94DB0A8093E80386E060E00E940D
:1022A000E10A87E061E00E94E10A89E06FE70E94AD
:1022B000E10A8AE065E00E94E10A8BE065E10E94A4
:1022C000E10A8CE062E10E94E10A8DE06DEF0E947C
:1022D000E10A8EE060E00E94E10A992019F084E1B1
:1022E00093E008C08091E50323E1829FC00111249F
:1022F0008B549D4F0E94060B80E36CE80E94E10A1C
:1023000082E36FE00E94E10A83E362E40E94E10A53
:1023100084E36AE00E94E10A85E36AE20E94E10A3E
:1023200086E36DE20E94E10A87E364ED0E94E10A20
:1023300088E360E00E94E10A89E360E00E94E10A2C
:10234000992049F0F5E7AF2EF1ECBF2EF1ECCF2E3E
:10235000FEEDDF2E08C0A090C703B090C803C09068
:10236000C903D090CA030AE38D2D9927AA27BB275A
:1023700089839A83AB83BC83802F69810E94E10AA1
:10238000802F8B5F69810E94E10ADC2CCB2CBA2C58
:10239000AA240F5F0E3341F783E46FEF0E94E10A36
:1023A00084E46FEF0E94E10A85E46FEF0E94E10A86
:1023B00086E46FEF0E94E10A992019F08DE666E04D
:1023C00003C08DE66091CB030E94E10A89E760E0DB
:1023D0000E94E10A8AE76091CC030E94E10A83E748
:1023E00060E00E94E10A84E760E00E94E10A99202F
:1023F00029F060EC72E98DEE99E108C06091C303A9
:102400007091C4038091C5039091C6030E94570B3D
:102410000F900F900F900F90CF91DF910F91DF9061
:10242000CF90BF90AF909F900895A0E0B0E0EBE117
:10243000F2E10C946A2F8CE00E94DB0A882379F584
:1024400085E296E063E171E00E94A72C5E9A80E04D
:102450000E9422110E94C10B5E9821C085E296E085
:102460000E94262E482F8091AD04882321F0842FCE
:102470000E94B80C14C080911805E82FF0E0319646
:102480009F012F71307031978091170590E02817C8
:10249000390729F0E251FB4F40832093180585E26C
:1024A00096E00E94EC2D892BC9F680919803843028
:1024B00009F08CC00E947A2960939C0470939D045B
:1024C00080939E0490939F04611571058105910589
:1024D00061F481E090E0A0E0B0E080939C049093F0
:1024E0009D04A0939E04B0939F048091A8049091B2
:1024F000A90481609093A9048093A80483E0809349
:1025000098038FE70E94B70AC5EED4E00E94CB0A79
:10251000899304E0CE3ED007C9F74091D004809162
:10252000E504282F30E0842F90E08227932786FF50
:1025300040C080E448274093D004C901887390705C
:10254000C89709F510E014C01F5F8091E603E12FE2
:10255000F0E084FF06C0EB51FB4F80810E94E40B4A
:1025600007C0EB51FB4F85E296E060810E945F2E31
:10257000212F30E08091E50490E087709070821701
:10258000930714F716C02F733070232B91F48091AA
:10259000E6048093A0048091E7048093A2048091D4
:1025A000E8048093A3048091EB048093AA04109222
:1025B000AB0480911905813019F482E080931905EC
:1025C00080911905833011F4109219050E947A291F
:1025D0005B016C018091A4049091A504A091A604D4
:1025E000B091A7040097A105B105C9F0A601950116
:1025F000281B390B4A0B5B0BDA01C901885B9B4036
:10260000A040B04060F00E94020B8093A1041092A1
:10261000A4041092A5041092A6041092A7048EEBB5
:1026200093E00E94160920919804309199044091FA
:102630009A0450919B0486017501E21AF30A040B77
:10264000150BE616F7060807190708F4EAC0A0926A
:102650009804B0929904C0929A04D0929B04A895D1
:102660008091AC04883008F0D4C08091AC048F5FB6
:102670008093AC04E0909C04F0909D0400919E0433
:1026800010919F04E114F1040105110511F18EEB85
:1026900093E00E941609AE18BF08C00AD10A6A1555
:1026A0007B058C059D0588F480919F0384FD04C003
:1026B00080ED97E00E940C0810929C0410929D04FB
:1026C00010929E0410929F0404C080E090E00E944B
:1026D0000C089091D004907C9093D0040091180540
:1026E000109117050117B1F180911905823091F50C
:1026F00090589093D0048EEB93E00E940C0989309F
:1027000010F048E002C0482F415030E013C03F5F56
:10271000A32FB0E0812F90E0FC01E251FB4F20811C
:10272000FD01E053FB4F2083A25FBA4F2C9301962B
:10273000182F1F71341710F4101749F7109317054D
:10274000832F895C9091D004892B8093D00430939F
:102750000E051AC0209119052430D1F490910E0570
:10276000EFE0F5E0A1EDB4E0292F30E02E0F3F1FA0
:1027700002C081918D93E217F307D9F7995C80919C
:10278000D004982B9093D00483E08093190523C044
:1027900080919304823029F491609093D0045E9AE2
:1027A0000FC09093D0045E98222319F481E08093A7
:1027B000190580911905833019F484E08093190577
:1027C000F8948091E603877067E273E041ED54E08E
:1027D0000E949D0978945D9A809192040E94EC0A6F
:1027E0008EEB93E00E940C09682F80ED94E00E942C
:1027F000B40EE0919204EF5FE0939204E83131F07F
:10280000F0E0E254FC4F8785882359F4109292043B
:1028100008C08091AC04883009F45E9A89E0809306
:10282000AC048091E603887171F180919803823045
:1028300051F58091A8049091A904880F991F909355
:10284000A9048093A80483E0809398030E94C10B9D
:102850000E947A296093A4047093A5048093A6042F
:102860009093A704611571058105910561F481E0DC
:1028700090E0A0E0B0E08093A4049093A504A0931E
:10288000A604B093A7048091E60384FF1EC0809144
:10289000A8049091A9048E7F0E945F0A182F80914E
:1028A000A0046091AA040E94A10C082F8091A104A9
:1028B000612F0E94A10C282F8091A2046091A30493
:1028C000402F009199030E9433105D9880919304EA
:1028D0008130C9F0813020F0823009F03FC033C030
:1028E0008EE00E949E2A892BC9F581E08093930493
:1028F0000E946C29609394047093950480939604CD
:10290000909397042BC08EE00E949E2A892B21F57C
:102910000E946C2920919404309195044091960472
:1029200050919704621B730B840B950B695E734087
:102930008040904098F082E08093930480ED97E08F
:102940000E940C080BC08EE00E949E2A892B31F059
:1029500080E090E00E940C0810929304CDB7DEB79F
:10296000EAE00C94862FACE1B0E0E9EBF4E10C94E2
:102970006A2F0E947A297B018C0181E00E9422113A
:1029800094E7A92E6E010894C11CD11C83E0B82ED7
:10299000A982C60161E00E94F00EB09298030E94E5
:1029A000C10B6AEF70E080E090E00E94A029809166
:1029B0009803833009F07DC085E296E00E94EC2DFB
:1029C000892B09F076C00E947A296E197F09800B45
:1029D000910B6058734C894C914008F06AC0D8CF75
:1029E0008FE70E94B70A0E94CB0A843509F05CC0C9
:1029F00089830E94CB0A182F00E010937A04009379
:102A000079040E94CB0A080F111D10937A040093D9
:102A100079040E94CB0A809378040E94CB0A8093A9
:102A20007704813108F040C0FF2407C00E94CB0A20
:102A3000095A1B4FF8018083F3940F2D10E0809109
:102A4000770490E0880F991F0817190778F380E73B
:102A50008983CE01019661E00E94F00E83E08093AD
:102A600098030E94C10B62E370E080E090E00E9456
:102A7000A029809198038330A9F08FE70E94B70ABC
:102A80000E94CB0A803581F4898303EA13E00E9417
:102A9000CB0AF80181938F01F3E00E3B1F07B9F7D2
:102AA00081E003C082E001C083E06C96EAE00C9410
:102AB000862F80919803833009F092CFF3CF0F9344
:102AC0001F93082F17C05E9A64E670E080E090E0E4
:102AD0000E94A0295E9864E670E080E090E00E9489
:102AE000A0291F5F101778F36CE271E080E090E09E
:102AF0000E94A02910E0F6CF482F392F25E00DC005
:102B0000F999FECF1FBA842F932F92BD81BD60BD6E
:102B10000FB6F894FA9AF99A0FBE215059F0F99924
:102B2000FECF842F932F92BD81BDF89A80B5681790
:102B300039F7089582E00E945F150895A0E0B0E0A3
:102B4000E4EAF5E10C94632F482E562EEE24FF2480
:102B500088249924C0E0D0E0CC24DD24E6E33E2E96
:102B600004C055245394CC24DD24442069F480917E
:102B70009903839DE00111247AE9E72E73E0F72E93
:102B800069E0862E912C1DC021E0421671F48091DF
:102B90009903839DE00111242B965EEBE52E53E013
:102BA000F52E49E2842E912C0CC032E0431649F4F4
:102BB00039E9E32E33E0F32E21E0822E912CC8ED8B
:102BC000D0E03E016C0C7D1C109222051092210574
:102BD000E3011BC0552059F4F999FECFD2BDC1BD08
:102BE000F89A80B5F701E00FF11F808307C0F70165
:102BF000E00FF11FCE0160810E947C150E0D1F1D9C
:102C0000F80180810E945C0821969E012619022FFE
:102C100010E008151905F0F2CE015520D9F4F99904
:102C2000FECFD2BDC1BDF89A20B5F999FECF21964D
:102C3000D2BDC1BD2197F89A80B590E0B22EAA24EA
:102C40008A299B29209121053091220528173907CF
:102C500059F487CF2196609122050E947C15CE0100
:102C6000609121050E947C1580E091E0C80ED91E7C
:102C700091E0C91693E0D90608F477CF852DCDB73A
:102C8000DEB7E1E10C947F2F80E061E00E949E15A9
:102C900081E061E00E949E15089580E060E00E945E
:102CA0009E15882331F081E060E00E949E15882304
:102CB00031F40E94BE080E9479080E9444160895CB
:102CC00082E061E00E949E15089582E060E00E942B
:102CD0009E1580919903843020F0109299030E94F0
:102CE000601608951F93182F0E946516809199030E
:102CF000811731F0143020F4109399030E9460166C
:102D00001F9108951092550485E6E0EFF3E0DF018E
:102D10001D928A95E9F708951F93182F8F3711F0A8
:102D20008830E1F5E0915504EE2309F455C0E150F7
:102D3000E0935504F0E0E051FC4F108285E296E00C
:102D40006DE00E945F2E10E00AC0E12FF0E0E0513C
:102D5000FC4F85E296E060810E945F2E1F5F8091AC
:102D60005504181790F385E296E060E20E945F2E0A
:102D700085E296E06DE00E945F2E10E00AC0E12F30
:102D8000F0E0E051FC4F85E296E060810E945F2E0A
:102D90001F5F80915504181790F31CC08B3119F4F4
:102DA0000E9482161FC08D30E9F08A30D9F08091E0
:102DB0005504843688F485E296E0612F0E945F2EE8
:102DC00080915504E82FF0E0E051FC4F10838F5FB5
:102DD0008093550480E007C085E296E067E00E949A
:102DE000132BF8CF81E01F9108951F93CF93DF93AA
:102DF000CDECD3E010E03BC085E296E062E271E00A
:102E00000E94A42C85E296E0612F4AE050E00E94E7
:102E1000212C85E296E06FE271E00E94A42C69917A
:102E200070E080E090E02091CC0330E040E050E0A2
:102E30000E94F32E20E137E240E050E00E94F32EA2
:102E4000DC01CB014091C3035091C4036091C503E1
:102E50007091C603480F591F6A1F7B1F85E296E0D9
:102E60002AE030E00E94E82B1F5F183119F08881BA
:102E7000882311F6DF91CF911F910895EF92FF9271
:102E80000F931F93882339F485E296E061E77AE097
:102E90000E94312B3BC090E00E94D30824E630E032
:102EA00040E050E00E94252F122F032FF42EE52E34
:102EB000622F732F842F952F2AE030E040E050E0FE
:102EC0000E94252F85E296E0BA01A9012AE030E0B0
:102ED0000E94D92B85E296E06EE20E94132B612FAF
:102EE000702F8F2D9E2D2AE030E040E050E00E94B0
:102EF000252FAB01BC0185E296E02AE030E00E947C
:102F0000D92B85E296E063E70E94452B1F910F9134
:102F1000FF90EF900895FF920F931F93CF93DF934D
:102F200085E296E067E67AE00E94F22A8091A303A8
:102F3000813041F485E296E06EE47AE00E94312B24
:102F4000FF246DC0823029F485E296E067E37AE0E1
:102F5000F5CF843029F485E296E063E27AE0EECFA3
:102F6000853071F785E296E068E17AE0E7CFCF2D12
:102F7000D0E0C930D1051CF06F2D685C02C06F2D08
:102F80006F5C85E296E00E94132B85E296E060E19B
:102F90007AE00E94F22ABE016F5F7F4F85E296E0E1
:102FA0004AE050E00E947D2C85E296E065E07AE000
:102FB0000E94F22A8E010D551C4FD8011196EC91FA
:102FC000E032F8F485E296E068EF79E00E94F22AB8
:102FD000F8018181803130F085E296E063E371E0B1
:102FE0000E94A42CCD55DC4F698170E06F70707029
:102FF0006F5F7F4F85E296E04AE050E00E94902CA0
:103000000DC0F0E0EF70F070EE0FFF1FE85BFC4FBB
:103010006081718185E296E00E94A72CF3948091F3
:103020007804F81608F4A3CF85E296E06DED79E018
:103030000E94F22A8091BB030E943E1785E296E02F
:1030400062EC79E00E94F22A8091BC030E943E1754
:1030500085E296E067EA79E00E94F22A8091BD035A
:103060000E943E1785E296E06CE879E00E94F22A21
:103070004091B3035091B4036091B5037091B603CE
:10308000411551056105710539F185E296E02AE0A7
:1030900030E00E94E82B85E296E069E579E00E9445
:1030A000F22A8091B7030E940609AB01BC0185E2B8
:1030B00096E02AE030E00E94E82B85E296E065E3A6
:1030C00079E00E94F22A85E296E06091B8034AE036
:1030D00050E00E94332C06C085E296E06CE279E075
:1030E0000E94312B85E296E06FE079E00E94F22A9F
:1030F0006091B9037091BA0385E296E04AE050E02E
:103100000E940D2C85E296E062EF78E00E94F22AA0
:103110006091B203603150F470E06F5F7F4F85E2E1
:1031200096E04AE050E00E94902C06C085E296E0CE
:1031300069EE78E00E94312B85E296E06CEC78E055
:103140000E94F22A8091B10380FD03C065E371E023
:1031500002C069E371E085E296E00E94A72C85E257
:1031600096E06FEA78E00E94F22A8091B1038270C3
:103170000E94AC0C85E296E060E978E00E94F22AB9
:103180008091B10384700E94AC0C85E296E061E707
:1031900078E00E94F22A8091B10388700E94AC0C02
:1031A000CDB7DEB7E5E00C948B2F1F93CF93DF9361
:1031B00085E296E06BEB7BE00E94F22A4091C3032C
:1031C0005091C4036091C5037091C60385E296E0F7
:1031D0002AE030E00E94E82B85E296E065EA7BE099
:1031E0000E94F22A4091C7035091C8036091C9031D
:1031F0007091CA0385E296E020E130E00E94E82B5E
:1032000085E296E06FE87BE00E94F22A85E296E094
:103210006091CB034AE050E00E94332C85E296E0B7
:1032200069E77BE00E94F22A85E296E06091CC0398
:103230004AE050E00E94332C85E296E063E67BE0B2
:103240000E94F22ACDECD3E010E012C0112331F03D
:1032500085E296E06DE371E00E94A42C85E296E0A1
:1032600069914AE050E00E94212C1F5F183119F04B
:103270008881882359F785E296E00E941B2B85E21E
:1032800096E06DE47BE00E94F22A85E296E0609190
:10329000E5034AE050E00E94332C85E296E068E3C3
:1032A0007BE00E94F22AE091E603F0E0E770F07024
:1032B000EE0FFF1FE859FC4F6081718185E296E0B7
:1032C0000E94A72C85E296E063E27BE00E94F22A4E
:1032D0008091E60390E0887190708830910589F0C4
:1032E000893091051CF4892B39F01BC08031910580
:1032F00069F04897B1F40FC085E296E06AE17BE09F
:103300000EC085E296E06EE07BE009C085E296E0C3
:1033100068E07BE004C085E296E06EEF7AE00E9410
:10332000312B85E296E06AEE7AE00E94F22A409123
:10333000BF035091C0036091C1037091C20385E245
:1033400096E02AE030E00E94E82B85E296E061ED0D
:103350007AE00E94F22A80919F0380710E94AC0C57
:1033600085E296E068EB7AE00E94F22A80919F0362
:1033700080740E94AC0C85E296E06FE97AE00E94CE
:10338000F22A80919F0380720E94AC0C85E296E045
:1033900062E87AE00E94F22A8EEB93E00E9416091E
:1033A000AB01BC0185E296E02AE030E00E94D92B17
:1033B00085E296E06DE77AE00E94F22A8EEB93E0D8
:1033C0000E9416099B01AC0160E472E48FE090E07A
:1033D0000E94252F85E296E0BA01A9012AE030E09B
:1033E0000E94D92B85E296E06AE77AE00E94312BB1
:1033F000DF91CF911F910895EF92FF920F931F934A
:103400007C0105E216E0C8016F2D70E04AE050E053
:103410000E94FC2BC8016EE20E94132BB70184E0CE
:10342000769567958A95E1F76F707070C8014AE0EC
:1034300050E00E94FC2BC8016EE20E94132B8FE02B
:10344000E822FF24C801B7014AE050E00E94FC2BAB
:103450001F910F91FF90EF9008950F931F93CF93BB
:10346000DF932091EF032F3FA9F585E296E061EF0E
:1034700075E00E94F22A84E693E00E94FC1985E23E
:1034800096E060ED75E00E94F22A809179049091B7
:103490007A040E94FC1985E296E06DE975E00E94CD
:1034A000312B85E296E06AE775E00E94312B85E2D8
:1034B00096E062E675E00E94312B85E296E06DE3CE
:1034C00075E00E94312B85E296E00E941B2B0E9442
:1034D0008B1769C012160CF066C0332727FD309594
:1034E0008091780490E0821793070CF45CC085E229
:1034F00096E068E275E00E94F22A6091EF03772778
:1035000067FD709585E296E04AE050E00E94902CBD
:1035100085E296E06DEF74E00E94F22A08E210E086
:103520003AC0C12FD0E0CC0FDD1FC95ADB4F288134
:1035300030E08091EF03992787FD90950197281738
:10354000390741F585E296E06FE371E00E94A42C13
:1035500085E296E0602F4AE050E00E94212C85E24F
:1035600096E063E471E00E94A42CE981F0E0EF7042
:10357000F070EE0FFF1FE85BFC4F6081718185E208
:1035800096E00E94A42C85E296E067E471E00E9438
:10359000A42C0F5F1F5F80917704181710F285E24B
:1035A00096E00E941B2BDF91CF911F910F91089500
:1035B000ACE1B0E0EEEDFAE10C946C2F282F809195
:1035C000EF038F3F09F042C1822F90E0FC013A9750
:1035D000EF36F10508F033C1EC5CFF4F0C94992FE6
:1035E00085E296E069E471E0AEC085E296E069E4C8
:1035F00071E00E94A72C1CC185E296E065E571E0B0
:103600000E94A72C85E78983DE011296E3EAF3E0A6
:103610008BE101900D928150E1F7CE0101966CE1B2
:103620000E94F00E0E94C10B83E08093980368EC27
:1036300070E080E090E00E94A0298091980384309F
:1036400009F0FDC08FE70E94B70A0E94CB0A898368
:10365000853509F0F4C085E296E06FED74E00E94D4
:10366000312B85E296E061EC74E00E94312B85E21B
:1036700096E063EA74E0ACC085E296E06DE671E046
:103680000E94A72C89E68983CE01019661E00E9401
:10369000F00E0E94C10B83E08093980368EC70E009
:1036A00080E090E00E94A02980919803843009F086
:1036B000C6C08FE70E94B70A0E94CB0A89838E0199
:1036C0000E5F1F4FBDE1EB2EF12CEC0EFD1E0E9494
:1036D000CB0AD8018D938D01AE15BF05C1F7A3EAC2
:1036E000B3E0FE0132968BE101900D928150E1F73B
:1036F0008981893409F0A3C085E296E065E874E029
:103700000E94312B85E296E067E674E00E94312B3F
:1037100085E296E069E474E05BC085E296E067E8E4
:1037200071E00E94A72C8EEF8093EF0388C0205297
:103730002750922F905380917804891738F485E2AE
:1037400096E066E971E00E94A72C79C09093EF03A0
:103750006FC084E18093EF0385E296E062E174E05C
:1037600037C085E18093EF0385E296E06BED73E06F
:103770002FC086E18093EF0385E296E064EA73E070
:1037800027C087E18093EF0385E296E06AE573E066
:103790001FC088E18093EF0385E296E069E473E05F
:1037A00017C089E18093EF0385E296E065E373E05B
:1037B0000FC08AE18093EF0385E296E060E273E058
:1037C00007C08BE18093EF0385E296E068EF72E03B
:1037D0000E94312B34C085E296E06EED72E00E94CB
:1037E000312B8091B10391E01DC085E296E068EC39
:1037F00072E00E94312B8091B10392E013C085E208
:1038000096E063EB72E00E94312B8091B10394E06B
:1038100009C085E296E068E972E00E94312B809150
:10382000B10398E089278093B1038FEF8093EF0372
:103830000E942D1A04C085E296E00E94262E85E2A1
:1038400096E00E94EC2D892BB1F762C1822F0E9475
:103850008C16882309F45CC180915504882321F4D7
:103860008FEF8093EF034CC180EF93E060E070E056
:1038700040E050E00E94A2069B01AC016091EF0382
:10388000862F992787FD9095A92FB92FFC01319795
:10389000EB31F10508F024C1ED55FF4F0C94992F41
:1038A000E62FFF27E7FDF0958091780490E08E17D2
:1038B0009F070CF415C1DA01C9010197A109B109EB
:1038C0008097A105B10548F0A8E2FA2E00E010E0CB
:1038D0006F010894C108D10825C0ED55FC4F822F17
:1038E00081508083E5C0612F70E0660F771F695AB1
:1038F0007B4FFB01808190E08C159D0591F48F2D0D
:1039000090E0A0E0B0E082179307A407B50741F468
:10391000F601ED55FC4FDB0111968C91818301E09E
:10392000F3941F5F809177041817E8F2BFC02F3F10
:1039300031054105510511F008F0D2C02093BB03B9
:10394000B7C02F3F31054105510511F008F0C8C03F
:103950002093BC03ADC02F3F31054105510511F047
:1039600008F0BEC02093BD03A3C08091F003806225
:10397000803719F581EF93E060E070E040E050E0BF
:103980000E94A2069B01AC01DC01CB010197A109B9
:10399000B1090897A105B10508F0B5C0CA01B90180
:1039A00024ED30E340E050E00E94F32E9B01AC0197
:1039B0002A5E3C4A4A46554E24C0863611F581EFB0
:1039C00093E060E070E040E050E00E94A2069B01BE
:1039D000AC01DC01CB010197A109B1090797A10551
:1039E000B10508F090C0CA01B90128EA31E640E00B
:1039F00050E00E94F32E9B01AC01245E3C434E46F6
:103A0000544E211531054105510561F0DA01C90116
:103A10008054914EAD49B8418158904FAA4FB24061
:103A200008F05EC02093B3033093B4034093B50312
:103A30005093B6033DC02F3F31054105510511F0AC
:103A400008F04EC02093B70333C0DA01C9010197D3
:103A5000A109B1098F3F9105A105B10508F040C04A
:103A60002093B80325C0DA01C901845C9940A040C5
:103A7000B0408D549D41A040B04030F43093BA0323
:103A80002093B90301E001C000E021153105410593
:103A9000510511F48FEF07C0213131054105510562
:103AA00028F4822F81508093B20302C00023C1F01A
:103AB000809156048823D1F48091C7039091C80364
:103AC000A091C903B091CA030196A11DB11D8093B5
:103AD000C7039093C803A093C903B093CA0306C059
:103AE00085E296E068EA71E00E94A72C0E948216A7
:103AF0008FEF8093EF0385E296E06AE00E94452B0A
:103B00000E942D1A05C021E030E040E050E07ECF59
:103B10006C96E8E00C94882F85E296E06CE472E005
:103B20000E94312B85E296E064E372E00E94312B23
:103B300085E296E00E94EC2D892B31F085E296E03B
:103B40000E94262E0E94D81A0E94B314823019F0C7
:103B5000833069F405C085E296E066E172E004C056
:103B600085E296E06FEF71E00E94312B08958FEFB0
:103B70008093EF03109256040E942D1A0CC085E228
:103B800096E00E94EC2D892B31F085E296E00E94B0
:103B9000262E0E94D81A8091EF038E3F81F7089558
:103BA0008091EF03992787FD9095A92FB92FFC01EC
:103BB0003196EB30F10508F074C0E254FF4F0C94DD
:103BC000992F85E296E064E678E00E94312B84E646
:103BD00093E00E94FC1985E296E06CE478E00E9494
:103BE000312B85E296E067E278E00E94312B85E296
:103BF00096E06DEF77E00E94312B85E296E06CED68
:103C000077E00E94312B85E296E06FEA77E00E9430
:103C1000312B85E296E069E877E00E94312B85E25E
:103C200096E065E677E00E94312B85E296E06EE350
:103C300077E00E94312B85E296E00E941B2B0E94C8
:103C4000D5182FC085E296E061E277E028C085E2D2
:103C500096E06CEF76E023C085E296E067EE76E0D2
:103C60001EC085E296E068EC76E019C085E296E039
:103C700064E876E014C085E296E06FE676E00FC077
:103C800085E296E06AE576E00E94312B85E296E0D7
:103C900064E176E004C085E296E06EEF75E00E9494
:103CA000312B6AE070E080E090E00E94A02904C01F
:103CB00085E296E00E94262E85E296E00E94EC2D99
:103CC000892BB1F70895A2E2B0E0E9E6FEE10C9499
:103CD000622F8E010F5F1F4F80E1D8011D928A95E0
:103CE000E9F785E296E066EC71E00E94A72C0E945D
:103CF0000A1120E431EE4DE958E12F8F38A349A392
:103D00005AA380EC91EDA8E9BBE18B8F9C8FAD8F1E
:103D1000BE8F24EF31E040E050E02F8B388F498F89
:103D20005A8F30E5C32E33ECD32EE12CF12C20E456
:103D3000422E21EE522E2DE9622E28E1722E882489
:103D40009924540133241E8A1D8A198A1A8A1B8ACF
:103D50001C8AFFC085E296E00E94262E8434B9F0CA
:103D6000853430F48332B9F18C3209F0CCC044C0D0
:103D7000833509F0C8C02F8D38A149A15AA1C901C6
:103D8000DA012C013D01882499245401E2C085E226
:103D900096E064E40E94132B85E296E040E451EE45
:103DA0006DE978E12AE030E00E94472C85E296E058
:103DB0006CE20E94132B85E296E040EC51ED68E93D
:103DC0007BE12AE030E00E94472C85E296E06CE23D
:103DD0000E94452BBEC019821A821B821C821D8242
:103DE0001E821F82188619861A861B861C861D86CF
:103DF0001E861F86188A3AC0339434E0331609F0C1
:103E0000A8C069817A818B819C8128EE33E040E0F3
:103E100050E00E94F32E6F8F78A389A39AA36D813F
:103E20007E818F8198850E94F32E6B8F7C8F8D8F82
:103E30009E8F89859A85AB85BC858F8B988FA98F3E
:103E4000BA8F6D857E858F8598890E94F32E6B01D0
:103E50007C0190E2C9169EE4D90690E0E90690E064
:103E6000F90630F48CE162E30E94E10A332471C068
:103E7000A0E3CA16A5E7DA06A0E0EA06A0E0FA0683
:103E800018F48CE162E2F0CFB0E4CB16BCE9DB06BB
:103E9000B0E0EB06B0E0FB0618F48CE166E2E4CF9C
:103EA000E0E5CE16E3ECDE06E0E0EE06E0E0FE063E
:103EB00018F48CE162E1D8CFF0E6CF16FAEEDF0617
:103EC000F0E0EF06F0E0FF0618F48CE165E1CCCFFE
:103ED00020E7C21621E1D20621E0E20620E0F20648
:103EE00018F48CE161E0C0CF30EAC31636E8D3069F
:103EF00031E0E30630E0F30618F48CE163E0B4CF80
:103F00008CE165E0B1CF90ED292E280E49E04215F5
:103F100000F1032D10E0000F111F000F111F81E0B1
:103F200090E08C0F9D1F080F191FD8016D917D9196
:103F30008D919C912AE030E040E050E00E94F32E09
:103F4000620D711D811D911DF80160837183828353
:103F5000938385E296E00E94EC2D892B09F0FACE3E
:103F600081149104A104B10489F4C301B2010E9437
:103F7000570B61E070E080E090E00E94A029FFEF25
:103F8000FE8B1D8A198A1A8A1B8A1C8A2F89388DF2
:103F9000498D5A8D82169306A406B506E0F40E9458
:103FA000020B29893A894B895C89280F311D411DF3
:103FB000511D298B3A8B4B8B5C8B3D89381708F44C
:103FC0008D8B4E89841708F48E8B0894811C911C6C
:103FD000A11CB11C56C0C301B20128EE33E040E081
:103FE00050E00E94252F85E296E0BA01A9012AE05F
:103FF00030E00E94D92B85E296E06CE20E94132B00
:1040000085E296E06D894AE050E00E94212C85E22D
:1040100096E06CE20E94132B69897A898B899C89CE
:10402000A50194010E94252F85E296E0BA01A9011D
:104030002AE030E00E94D92B85E296E06CE20E94F3
:10404000132B85E296E06E894AE050E00E94212C15
:1040500085E296E06CE20E94452B4C0C5D1C6E1CC8
:104060007F1C8B8D9C8DAD8DBE8D84159505A60511
:10407000B70520F44F8C58A069A07AA08824992411
:1040800054012F8D38A149A15AA1285E33404040E8
:10409000504009F05ECFA296E2E10C947E2FAAE593
:1040A000B0E0E5E5F0E20C946E2F8B017A018B30E5
:1040B00009F425C18C3040F5853009F484C0863080
:1040C00080F4823009F459C0833020F4813009F043
:1040D00058C242C0833009F461C0843009F051C233
:1040E00065C0883009F49DC0893038F4863009F401
:1040F00086C0873009F045C28CC0893009F499C068
:104100008A3009F03EC2C9C0893609F48AC18A36AC
:1041100080F4863609F435C1873620F4853609F0F7
:1041200030C216C1873609F445C1883609F029C264
:1041300049C18C3609F4CCC18D3638F48A3609F47D
:104140007BC18B3609F01DC2B7C18D3609F4F4C1AD
:10415000873C09F016C208C281E069E270E00E9463
:10416000A8100EEB13E0F80181918F010E949110CD
:10417000F3E0073E1F07B9F70CC282E06BE170E085
:104180000E94A81003EA13E0F80181918F010E94B8
:104190009110F3E00E3B1F07B9F7FBC183E061E02C
:1041A00070E00E94A8100E94B314F1C184E061E0A5
:1041B00070E00E94A81081E00E9491100E948A1075
:1041C0000E94631EE8C16091770470E0660F771F5C
:1041D00085E00E94A81000E010E008C0F801E95A4C
:1041E000FB4F80810E9491100F5F1F4F80917704D9
:1041F00090E0880F991F0817190780F3CAC186E05D
:1042000062E070E00E94A81084E693E00E949F1094
:10421000C0C187E061E070E00E94A810809178043E
:10422000B6C188E061E070E00E94A8108091990317
:10423000AEC186E68983CE01019661E00E94F00E50
:104240000E94C10B83E08093980368EC70E080E0EB
:1042500090E00E94A029809198038430E1F48FE7D8
:104260000E94B70A0E94CB0A8983863471F489E0E0
:1042700060E270E00E94A81010E00E94CB0A0E9449
:1042800091101F5F1032C9F784C189E061E070E0CE
:104290000E94A810CFC089E075C18AE069E070E093
:1042A0000E94A81010929A0380918F05882351F0E4
:1042B00080919F039091A003A091A103B091A203CC
:1042C000806809C080919F039091A003A091A103F1
:1042D000B091A2038F7780939F039093A003A09344
:1042E000A103B093A2030AE913E0F80181918F01C1
:1042F0000E949110F3E0033A1F07B9F74AC18BE01F
:1043000061E270E00E94A8108091AC048F3F39F008
:104310008091AC048F5F8093AC04815002C0809187
:10432000AC040E94911000E010E0F894F801EE0F48
:10433000FF1FE95DFC4F808191810E943A0A0E9433
:104340009F1078940F5F1F4F0031110571F721C145
:1043500085E661E070E00E94A8100932110509F0BD
:1043600015C120E030E0F901E254FC4FD701A20F63
:10437000B31F8C9180832F5F3F4F2932310599F70E
:1043800059C086E661E070E00E94A8100B3111056B
:1043900009F0FCC020E030E0F901ED55FC4FD701F9
:1043A000A20FB31F8C9180832F5F3F4F2B313105BC
:1043B00099F740C087E661E070E00E94A8100E9473
:1043C000441638C088E661E070E00E94A81085E7D6
:1043D0008A83DE011396E3EAF3E08BE101900D920C
:1043E0008150E1F7CE0102966CE10E94F00E0E942E
:1043F000C10B83E08093980360E273E080E090E07B
:104400000E94A02980919803843009F0BFC08FE7F3
:104410000E94B70A0E94CB0A8A83853509F0B6C08C
:1044200009C089E661E070E00E94A8100E94790846
:104430000E94BE0881E0ABC08AE661E070E00E94A5
:10444000A81089E68E8FCE014E9661E00E94F00E94
:104450000E94C10B83E08093980360E273E080E0E8
:1044600090E00E94A02980919803843009F08EC0CA
:104470008FE70E94B70A0E94CB0A8E8F8E01015EE1
:104480001F4F4AE3E42EF12CEC0EFD1E0E94CB0AD6
:10449000F80181938F01EE15FF05C1F7A3EAB3E0A0
:1044A000FE017F968BE101900D928150E1F78E8D98
:1044B000893409F06BC0BECF8BE661E070E00E94EA
:1044C000A810F70180810E9472160E944D16B2CF8B
:1044D0008CE661E070E00E94A8100032110571F4D2
:1044E00087E68AAFDE01DB96F70180E201900D924C
:1044F0008150E1F7CE01CA9661E205C087E48AAF38
:10450000CE01CA9661E00E94F00E0E94C10B83E0CA
:10451000809398036CE474E080E090E00E94A0290E
:1045200080919803843091F58FE70E94B70A0E942A
:10453000CB0A873459F57ECF8DE661E070E00E94AA
:10454000A8100930110511F520E030E0F901E65618
:10455000FC4FD701A20FB31F8C9180832F5F3F4F79
:104560002930310599F766CF87EC61E070E00E9451
:10457000A81081E00E9491100E948A101092ED0311
:104580000AC08AEC61E070E00E94A81080E00E94FE
:1045900091100E948A10C65ADF4FE6E00C948A2FD1
:1045A000A0E0B0E0E6EDF2E20C946A2F84E0A82EE1
:1045B00006E0B02E15E0C12E03E215E0B4E6DB2ED6
:1045C000A2E0EA2EF3E0FF2EA1C085E296E00E9471
:1045D000262E982F80938E0580918D05833021F1B2
:1045E000843028F4813099F08230B8F409C08530E5
:1045F00009F448C0853020F1863009F087C05FC0DB
:10460000953B09F083C081E080938D057FC0923691
:1046100009F07AC0E0928D0579C090938C05909353
:104620008B05F0928D0572C09093890510928A05D2
:1046300080918B05892780938B05A0928D0566C09C
:10464000D92FC0E02091890530918A052C2B3D2B74
:1046500030938A052093890580918B058927809363
:104660008B05C0928D052536310508F44FC08CECC2
:1046700061E070E00E94A81081E00E9491100E9409
:104680008A1042C02091870530918805F901ED5DBF
:10469000FA4F908380918B05892780938B052F5F3C
:1046A0003F4F30938805209387058091890590912D
:1046B0008A052817390750F1B0928D0527C08091DF
:1046C0008B05891759F46091870570918805809151
:1046D0008C0543E255E00E944F200DC08BEC62E058
:1046E00070E00E94A81080918C050E94911080912A
:1046F000EE030E949110F8018D2D11928A95E9F731
:10470000109288051092870510928D0585E296E03B
:104710000E94EC2D892B09F058CFCDB7DEB7EAE027
:104720000C94862F81E08093ED0308C085E296E02B
:104730000E94EC2D892B11F00E94D0228091ED0374
:104740008823A1F70895A0E0B0E0E9EAF3E20C9431
:104750006D2F0E947A296115710581059105C9F3B4
:104760000E9499061092C7031092C8031092C903C1
:104770001092CA03DD24E090C703F090C8030091B3
:10478000C9031091CA03102F0F2DFE2CEE240E9496
:1047900094062FEF30E040E050E00E94472FE60EF5
:1047A000F71E081F191FE092C703F092C803009379
:1047B000C9031093CA03D39444E0D416E1F6CDECB8
:1047C000D3E000E010E090E1E92E97E2F92E4EC030
:1047D0000F5F19F40E9479084DC00E94940622E3ED
:1047E00030E040E050E00E94472F6F5FEDECF3E0D7
:1047F00090E004C08191861759F39F5F9117D0F321
:104800008091CC0390E08E9D90018F9D300D9E9DF8
:10481000300D1124862F90E0AC01249FC001259F0C
:10482000900D349F900D1124AA2797FDA095BA2FC3
:104830002091C3033091C4034091C5035091C60336
:10484000820F931FA41FB51F20919B0330919C03DF
:1048500040919D0350919E03281739074A075B0733
:1048600008F4B6CF69931F5F183121F0888188233F
:1048700009F0AECFCDB7DEB7E7E00C94892F1F93D8
:104880001091EF031F3F09F0F1C0893409F467C0AC
:104890008A3428F5883309F479C0893368F4803381
:1048A00009F486C0813308F06FC08B3109F44DC024
:1048B000813209F0D5C03DC0813409F49AC08234F8
:1048C00038F4893309F472C0803409F0C9C031C0AA
:1048D000823409F4A1C0863409F0C2C052C08236C5
:1048E00009F49AC0833690F4883579F1893538F423
:1048F000823509F43FC0833509F0B2C01FC08A3544
:1049000009F4A9C0813609F0ABC073C0823791F1B8
:10491000833730F48636A9F1893609F0A1C01FC06B
:10492000883799F08A3709F496C0833709F098C020
:1049300005C085E296E069E471E019C00E94441662
:1049400085E296E063ED71E006C00E944D1685E2B7
:1049500096E06DEE71E00E94A72C8EEF7FC00E9462
:1049600079080E94BE0885E296E06CE072E00E9441
:10497000A72C76C00E94A32385E296E065E272E050
:10498000F6CF0E94F5166CC0805368C085E296E0B1
:104990006CEE71E00E94312B9091E603892F885FC5
:1049A0008871977E892B8093E60320C089E056C0EA
:1049B00085E296E069ED71E00E94312B80919F03C2
:1049C0009091A003A091A103B091A20320E130E057
:1049D00040E050E082279327A427B52780939F03C8
:1049E0009093A003A093A103B093A2031093EF03AD
:1049F00037C085E296E063EC71E00E94312B809134
:104A00009F039091A003A091A103B091A20320E481
:104A100030E040E050E012C085E296E062EB71E0E9
:104A20000E94312B80919F039091A003A091A1033C
:104A3000B091A20320E230E040E050E082279327CB
:104A4000A427B52780939F039093A003A093A1036D
:104A5000B093A20302C00E948C1D8FEF8093EF03DE
:104A60008091EF038E3F09F4DDC0D4C00E948C1604
:104A7000882309F4D7C080915504882321F48FEF4F
:104A80008093EF03C7C080EF93E060E070E040E008
:104A900050E00E94A2069B01AC018091EF03992790
:104AA00087FD9095A92FB92FFC013197E930F105C9
:104AB00008F08CC0E753FF4F0C94992FDA01C9011D
:104AC0008154914EAD49B8418F57904FAA4FB24093
:104AD00008F07CC02093C3033093C4034093C50304
:104AE0005093C6039AC02093C7033093C8034093E2
:104AF000C9035093CA0381E0809356048EC02830C6
:104B000031054105510508F061C02093CB0385C0F4
:104B1000DA01C9010197A109B1090A97A105B105F7
:104B200008F054C02093CC0378C080EF93E06DE38D
:104B300071E00E94BE0710E00EC0183130F4E12F82
:104B4000F0E0E254FC4F87871F5F80E090E06DE368
:104B500071E00E94BE07009759F00E94A0070097DD
:104B600061F706C0E12FF0E0E254FC4F17861F5FAB
:104B70001831C0F352C0253031054105510530F5DB
:104B80002093E5034AC0DA01C9010197A109B109DF
:104B90000697A105B105D0F48091E603887F822BAA
:104BA0008093E6033AC0DA01C9010197A109B1096E
:104BB0008050924CA140B04048F42093BF03309302
:104BC000C0034093C1035093C20327C085E296E01F
:104BD00068EA71E00E94A72C13C08091C7039091EE
:104BE000C803A091C903B091CA030196A11DB11DCC
:104BF0008093C7039093C803A093C903B093CA03DB
:104C00000E9482168FEF8093EF0385E296E06AE0C0
:104C10000E94452B0E94D01D05C080915604882318
:104C2000E1F2EECF1F9108958FEF8093EF03109282
:104C300056040E94D01D0CC085E296E00E94EC2D27
:104C4000892B31F085E296E00E94262E0E943F24B7
:104C50008091EF038E3F81F76AE070E080E090E0A2
:104C60000E94A02904C085E296E00E94262E85E2DB
:104C700096E00E94EC2D892BB1F70895AAE2B0E0EE
:104C8000E4E4F6E20C94672F0E946C297B018C010E
:104C900081E00E94221104C085E296E00E94262E47
:104CA00085E296E00E94EC2D892BB1F75E98DD2419
:104CB000D39452E6752E42E0842E912C8C0E9D1ECC
:104CC0005E010894A11CB11C33E0C32E0E946C2924
:104CD00020E030E06E197F09800B910B693C710573
:104CE0008105910510F021E030E08D2D90E0282322
:104CF0003923232B99F10E946C297B018C015D9A49
:104D000080ED97E00E940C087982D401EEEBF3E08D
:104D100089E201900D928150E1F7C5016AE20E949B
:104D2000F00E5D9880E090E00E940C08C09298031D
:104D30000E94C10B62E370E080E090E00E94A02935
:104D400080919803843051F4C09298038FE70E94B9
:104D5000B70A0E94CB0A823409F4DD248EE00E9457
:104D60009E2A892B49F5DD24D39426C05E9A5D9A4C
:104D700085E296E00E94262E8D30910569F08E30F6
:104D800091051CF40A97B1F407C08332910569F0CC
:104D90008234910579F40CC085E296E064EA71E012
:104DA0000E94312B0E94142605C00E94631E02C07F
:104DB0000E9492235E985D9885E296E00E94EC2D19
:104DC000892B09F483CFD2CF8F929F92AF92BF925B
:104DD000CF92DF92EF92FF920F931F938EE00E948B
:104DE0009E2A892B09F083C068EC70E080E090E097
:104DF0000E94A02980E090E00E940C080E946C298B
:104E00005B016C0160ECE62E62E1F62E012D112DA6
:104E1000EA0CFB1C0C1D1D1D06C08EE00E949E2A84
:104E2000892B09F062C00E946C296E157F058007EE
:104E3000910798F38EE00E949E2A892B09F055C0B5
:104E400080ED97E00E940C080E946C297B018C0188
:104E500099249394882488E496E2A0E0B0E0A80E18
:104E6000B91ECA1EDB1E29C0AE14BF04C006D1067F
:104E700038F480ED97E00E940C08882483941DC0CC
:104E80000E946C296E197F09800B910B693C71059A
:104E90008105910590F00E946C297B018C0180E0D6
:104EA000992009F481E0982E882319F480E090E09D
:104EB00002C080ED97E00E940C088EE00E949E2ABE
:104EC000892B91F280E090E00E940C08882049F044
:104ED000809199038F5F83700E9472160E944D1615
:104EE00006C00E94A3230E9444160E943E261F91E2
:104EF0000F91FF90EF90DF90CF90BF90AF909F9079
:104F00008F90089580E06DEF77E042E050E00E94DE
:104F1000A7280895EF92FF920F931F9380E00E94BD
:104F200045080E94C71089E061E00E94FF2989E0DE
:104F300060E00E946B2A86E061E00E94FF2985E024
:104F400061E00E94FF298EE060E00E94FF2988E076
:104F500060E00E94FF2988E061E00E946B2A81E105
:104F600061E00E94FF2981E160E00E946B2A0E94BB
:104F7000DC1085E296E040E052EC61E070E00E94D7
:104F8000652D0E9465160E944D160E94860C8FEFBB
:104F90008093AC040E94822778940E946C297B0144
:104FA0008C018091AC048F3F09F0C7C00E946C292E
:104FB0006E197F09800B910B605D774080409040B7
:104FC00008F0BBC0EECF85E296E00E94262E85E277
:104FD00096E00E94EC2D892BB1F785E296E062E421
:104FE00072E00E94A42C84E693E00E94FC1985E202
:104FF00096E069E572E00E94A42C85E296E064E008
:1050000070E04AE050E00E94902C62E370E080E0A3
:1050100090E00E94A02985E296E00E94EC2D049782
:105020000CF185E296E00E94262E82349105D1F49F
:1050300085E296E00E94262E8E34910599F485E251
:1050400096E00E94262E8434910561F485E296E074
:105050000E94262E819731F480E090E00E940C0897
:105060000E943E264091BF035091C0036091C1034E
:105070007091C203DB01CA010197A109B10904972C
:10508000A105B10568F44093AD04433029F040E038
:1050900052EC61E070E004C040EA56E861E070E084
:1050A00085E296E00E94652D0E94E4265E9880E0ED
:1050B00090E00E940C080E94860C80E00E94221161
:1050C000809192040E94EC0A0E94C10B1092170575
:1050D000109218051092190510E015C062E370E0F7
:1050E00080E090E00E94A02980ED97E00E940C08EB
:1050F00062E370E080E090E00E94A02980E090E010
:105100000E940C081F5F80919903811738F78091E6
:10511000E60390E084FF09C020E088719070489712
:1051200009F421E0822F0E94EB108FE00E944508D5
:105130001F910F91FF90EF90089580ED97E00E94EE
:105140000C088EE061E00E946B2A5E9A40CF8230AC
:1051500000F5E82FF0E0EE0FFF1FE057FA4F7183E4
:105160006083882319F08130A1F408C08091690020
:105170008C7F842B80936900E89A08958091690060
:10518000440F551F440F551F837F842B8093690064
:10519000E99A08951F920F920FB60F9211242F9340
:1051A0003F934F935F936F937F938F939F93AF93AF
:1051B000BF93EF93FF938091900590919105892B78
:1051C00029F0E0919005F09191050995FF91EF91FB
:1051D000BF91AF919F918F917F916F915F914F910F
:1051E0003F912F910F900FBE0F901F9018951F9217
:1051F0000F920FB60F9211242F933F934F935F930B
:105200006F937F938F939F93AF93BF93EF93FF938E
:105210008091920590919305892B29F0E091920558
:10522000F09193050995FF91EF91BF91AF919F91F7
:105230008F917F916F915F914F913F912F910F903F
:105240000FBE0F901F9018951F920F920FB60F92DE
:1052500011242F933F938F939F93AF93BF9380918C
:10526000980590919905A0919A05B0919B05309170
:105270009C050196A11DB11D232F2D5F2D3720F018
:105280002D570196A11DB11D20939C058093980573
:1052900090939905A0939A05B0939B0580919405EE
:1052A00090919505A0919605B09197050196A11D45
:1052B000B11D8093940590939505A0939605B093A6
:1052C0009705BF91AF919F918F913F912F910F9033
:1052D0000FBE0F901F9018958FB7F89420919805E6
:1052E0003091990540919A0550919B058FBFB90166
:1052F000CA0108959FB7F8942091940530919505BF
:10530000409196055091970586B5A89B06C08F3FA2
:1053100021F02F5F3F4F4F4F5F4F9FBF542F432FC1
:10532000322F2227280F311D411D511D82E0220FEF
:10533000331F441F551F8A95D1F7B901CA0108953B
:10534000EF92FF920F931F93CF93DF937B018C011A
:105350000E947A29EB010EC00E947A296C1B7D0BFA
:10536000685E7340C8F30894E108F1080109110967
:10537000C851DC4FE114F1040105110569F7CDB7FF
:10538000DEB7E6E00C948A2F789484B5826084BD01
:1053900084B5816084BD85B5826085BD85B5816039
:1053A00085BDEEE6F0E0808181608083E1E8F0E099
:1053B0001082808182608083808181608083E0E8C8
:1053C000F0E0808181608083E1EBF0E080818460A7
:1053D0008083E0EBF0E0808181608083EAE7F0E0A9
:1053E000808184608083808182608083808181600D
:1053F00080838081806880831092C1000895CF935C
:10540000DF93482F50E0CA018D5F934FFC01349128
:105410004151544FFA018491882369F190E0880F3B
:10542000991FFC01EF52F44FA591B491FC01E55294
:10543000F44FC591D491662351F42FB7F8948C9111
:10544000932F909589238C93888189230BC0623098
:1054500061F42FB7F8948C91932F909589238C93B6
:105460008881832B88832FBF06C09FB7F8948C91C7
:10547000832B8C939FBFDF91CF910895833071F080
:10548000843028F48130A1F0823021F514C08630B8
:10549000B1F08730D1F08430E9F404C0809180000D
:1054A0008F7703C0809180008F7D80938000089566
:1054B00084B58F7702C084B58F7D84BD08958091B7
:1054C000B0008F778093B00008958091B0008F7DF9
:1054D0008093B0000895FF920F931F93F62E482FEC
:1054E00050E0CA01895E934FFC012491CA018D5F8F
:1054F000934FFC0114914151544FFA010491002340
:10550000C9F0222319F0822F0E943E2AE02FF0E0FA
:10551000EE0FFF1FE552F44FA591B4919FB7F89499
:10552000FF2021F48C911095812302C08C91812B56
:105530008C939FBF1F910F91FF9008950F931F931E
:10554000482F50E0CA01895E934FFC012491CA01A3
:105550008D5F934FFC0104914151544FFA01149116
:10556000112319F420E030E015C0222319F0822F16
:105570000E943E2A812F90E0880F991F8B51944FF3
:10558000FC01A591B4918C9120E030E0802311F0D2
:1055900021E030E0C9011F910F910895A0E0B0E033
:1055A000E4EDFAE20C946C2F7C016B018A01C0E0FF
:1055B000D0E00FC0D6016D916D01D701ED91FC9146
:1055C0000190F081E02DC7010995C80FD91F015046
:1055D00010400115110571F7CE01CDB7DEB7E8E037
:1055E0000C94882FEF92FF920F931F93CF93DF932A
:1055F0007C018B01C0E0D0E0F8010F5F1F4F649188
:10560000662359F0D701ED91FC910190F081E02DD6
:10561000C7010995C80FD91FEFCFCE01CDB7DEB7AF
:10562000E6E00C948A2FDC01ED91FC910190F08171
:10563000E02D09950895EF92FF920F931F938C012F
:105640006DE00E94132B7C01C8016AE00E94132BBD
:105650009C012E0D3F1DC9011F910F91FF90EF90EE
:105660000895EF92FF920F931F937C010E94F22AFC
:105670008C01C7010E941B2B9C01200F311FC90107
:105680001F910F91FF90EF900895EF92FF920F936B
:105690001F937C010E94132B8C01C7010E941B2BBE
:1056A0009C01200F311FC9011F910F91FF90EF90B6
:1056B0000895CF93DF93EC016115710519F420E093
:1056C00030E00FC0DB010D900020E9F71197A61B19
:1056D000B70BE881F9810280F381E02DAD010995D6
:1056E0009C01C901DF91CF9108954F925F927F9203
:1056F0008F929F92AF92BF92CF92DF92EF92FF92E2
:105700000F931F93DF93CF93CDB7DEB7A1970FB65B
:10571000F894DEBF0FBECDBF2C01742ECB0122301A
:1057200008F42AE019A231E2C32ED12CCC0EDD1EE2
:10573000822E9924AA24BB24672D752FA5019401DC
:105740000E94252F79018A01C801B701A5019401A2
:105750000E94F32E472D461B0894C108D1084A30F9
:1057600010F4405D01C0495CF6014083E114F1048E
:105770000105110521F07E2C5F2DC801DDCFC2018E
:10578000B6010E94592BA1960FB6F894DEBF0FBE4A
:10579000CDBFCF91DF911F910F91FF90EF90DF90E0
:1057A000CF90BF90AF909F908F907F905F904F90E1
:1057B0000895DC012115310541F4ED91FC91019032
:1057C000F081E02D642F099508950E94752B0895AE
:1057D000EF92FF920F931F937C010E94D92B8C01B3
:1057E000C7010E941B2B9C01200F311FC9011F9173
:1057F0000F91FF90EF900895EF92FF920F931F93F8
:105800009A017B0100E010E0B801A7010E94D92BAA
:105810001F910F91FF90EF900895EF92FF920F93D9
:105820001F937C010E94FC2B8C01C7010E941B2B43
:105830009C01200F311FC9011F910F91FF90EF9024
:105840000895EF92FF920F931F939A01E62EFF2483
:1058500000E010E0B801A7010E94D92B1F910F9121
:10586000FF90EF900895EF92FF920F931F937C01AA
:105870000E94212C8C01C7010E941B2B9C01200F30
:10588000311FC9011F910F91FF90EF900895A0E083
:10589000B0E0EDE4FCE20C946C2FEC016A017B01BA
:1058A0002115310541F4E881F9810190F081E02D65
:1058B000642F09951BC02A303105B1F477FF13C05E
:1058C0006DE20E94132B8C0144275527BA014C1915
:1058D0005D096E097F09CE012AE00E94752B9C01AB
:1058E000200F311F04C02AE00E94752B9C01C901C2
:1058F000CDB7DEB7E8E00C94882FEF92FF920F93BC
:105900001F937B019A010027F7FC0095102FB80127
:10591000A7010E94472C1F910F91FF90EF900895CF
:10592000EF92FF920F931F937C010E947D2C8C01BC
:10593000C7010E941B2B9C01200F311FC9011F9121
:105940000F91FF90EF9008950E94592B0895EF92C8
:10595000FF920F931F937C010E94A42C8C01C7011E
:105960000E941B2B9C01200F311FC9011F910F9119
:10597000FF90EF90089508951F920F920FB60F9227
:1059800011242F933F934F938F939F93EF93FF9304
:105990008091C00082FD1DC04091C6002091DD05B0
:1059A0003091DE052F5F3F4F2F7330708091DF0500
:1059B0009091E0052817390771F0E091DD05F0912D
:1059C000DE05E356FA4F40833093DE052093DD0574
:1059D00002C08091C600FF91EF919F918F914F91EE
:1059E0003F912F910F900FBE0F901F9018951F920F
:1059F0000F920FB60F9211242F933F938F939F9383
:105A0000EF93FF9320912106309122068091230687
:105A1000909124062817390731F48091C1008F7DB9
:105A20008093C10014C0E0912306F0912406EF5149
:105A3000FA4F2081809123069091240601968F735E
:105A4000907090932406809323062093C600FF91C4
:105A5000EF919F918F913F912F910F900FBE0F90DB
:105A60001F901895A0E0B0E0E8E3FDE20C94682FE9
:105A7000FC011382128288EE93E0A0E0B0E0848300
:105A80009583A683B7838AE893E0918380837587A3
:105A9000648757874687318B208B138B028BF58A5F
:105AA000E48AD78AC68AB18EA08E938E828E8F8525
:105AB000848F8889858F8989868F8A89878F8B894A
:105AC00080A32096ECE00C94842FAF92BF92DF92DB
:105AD000EF92FF920F931F93CF93DF93EC017A0124
:105AE0008B01DD24403081EE580780E0680780E0BC
:105AF000780711F0DD24D39491E0A92EB12CEC8924
:105B0000FD89DD2069F0C50108A002C0880F991F3A
:105B10000A94E2F7808360E079E08DE390E005C0CD
:105B2000108260E874E88EE190E0A80197010E947D
:105B3000252F21503040404050405695479537958D
:105B4000279580E12030380720F0DD2011F0DD249A
:105B5000D6CFE889F9893083EA89FB89208319A2A5
:105B6000EE89FF89408121E030E0C9010C8C02C040
:105B7000880F991F0A94E2F7482B4083EE89FF892A
:105B80004081C9010D8C02C0880F991F0A94E2F769
:105B9000482B4083EE89FF894081C9010E8C02C0E9
:105BA000880F991F0A94E2F7482B4083EE89FF89FA
:105BB00080810F8C02C0220F331F0A94E2F72095D8
:105BC00028232083DF91CF911F910F91FF90EF90B9
:105BD000DF90BF90AF900895DC011C96ED91FC9191
:105BE0001D97E05CFF4F2191319180819181281BAD
:105BF000390B2F733070C901089585E296E00E9439
:105C0000EC2D892B11F00E94BB2C0895DC011C9611
:105C1000ED91FC911D97E05CFF4F20813181E054B4
:105C2000F040DF01AE5BBF4F8D919C91119728171B
:105C3000390719F42FEF3FEF07C08D919C91E80FC2
:105C4000F91F8081282F30E0C9010895DC011C96DE
:105C5000ED91FC911D97E05CFF4F20813181E05474
:105C6000F040DF01AE5BBF4F8D919C9111972817DB
:105C7000390719F42FEF3FEF10C08D919C911197C8
:105C8000E80FF91F20818D919C91119701968F73D8
:105C9000907011969C938E9330E0C9010895DC01B9
:105CA00091968C919197882339F05496ED91FC91BF
:105CB0005597808186FFF9CF91961C920895CF93D6
:105CC000DF93EC01EE85FF85E05CFF4F20813181A1
:105CD000E054F0402F5F3F4F2F733070DF01AE5B19
:105CE000BF4F8D919C91119728173907D1F3E05C34
:105CF000FF4F80819181E054F040E80FF91F6083ED
:105D0000EE85FF85E05CFF4F31832083EE89FF89BC
:105D1000208181E090E00F8C02C0880F991F0A94C7
:105D2000E2F7282B208381E089A3EC89FD8980811B
:105D30008064808381E090E0DF91CF9108958F921D
:105D40009F92AF92BF92CF92DF92EF92FF920F930A
:105D50001F9300D000D00F92EDB7FEB7319684E0CC
:105D6000ADB7BEB711968C9383E0818387E08283C1
:105D700085E0838381E0848385E296E06DE975E0C8
:105D800041EE55E025EC30E004EC10E0B0ECEB2EF9
:105D9000F12CA1ECCA2ED12CF2ECAF2EB12CE6ECFA
:105DA0008E2E912C0E94322D0F900F900F900F90FD
:105DB0000F901F910F91FF90EF90DF90CF90BF90C9
:105DC000AF909F908F900895CF93DF930E94C42946
:105DD0000E948A27CDEFDDE20E9415122097E1F3A1
:105DE0000E94FD2DF9CF629FD001739FF001829F29
:105DF000E00DF11D649FE00DF11D929FF00D839F5A
:105E0000F00D749FF00D659FF00D9927729FB00DF6
:105E1000E11DF91F639FB00DE11DF91FBD01CF0109
:105E20001124089597FB092E07260AD077FD04D088
:105E300086D006D000201AF4709561957F4F0895A2
:105E4000F6F7909581959F4F0895A1E21A2EAA1B0F
:105E5000BB1BFD010DC0AA1FBB1FEE1FFF1FA2171A
:105E6000B307E407F50720F0A21BB30BE40BF50B17
:105E7000661F771F881F991F1A9469F760957095A0
:105E8000809590959B01AC01BD01CF01089597FBD2
:105E9000092E05260ED057FD04D0D7DF0AD0001CEE
:105EA00038F450954095309521953F4F4F4F5F4FB7
:105EB0000895F6F790958095709561957F4F8F4F77
:105EC0009F4F08952F923F924F925F926F927F92D1
:105ED0008F929F92AF92BF92CF92DF92EF92FF92FA
:105EE0000F931F93CF93DF93CDB7DEB7CA1BDB0BA6
:105EF0000FB6F894DEBF0FBECDBF09942A8839884B
:105F000048885F846E847D848C849B84AA84B98451
:105F1000C884DF80EE80FD800C811B81AA81B9815D
:105F2000CE0FD11D0FB6F894DEBF0FBECDBFED0171
:105F30000895EE0FFF1F0590F491E02D0994AA1B20
:105F4000BB1B51E107C0AA1FBB1FA617B70710F064
:105F5000A61BB70B881F991F5A95A9F78095909596
:105F6000BC01CD010895911106C0803219F089500D
:105F70008550D0F70895992788270895F894FFCF82
:105F80004E6F005965730054582074696D656F75C4
:105F90007421006D6F64756C65206C6F636B656454
:105FA0003F00486F70206368616E6E656C20002052
:105FB00040200053004E2F4100386368002C002C15
:105FC000205B005D20280029004E4F5420454E41A3
:105FD000424C45440053656E64696E672073657476
:105FE00074696E677320746F2052580A005265738B
:105FF000657474696E672073657474696E67732065
:106000006F6E2052580A0041626F72746564206599
:10601000646974730A00696E76616C6964207365E3
:106020006C656374696F6E000D0A496E76616C6908
:106030006420696E707574202D20646973636172C9
:106040006465642107007363616E6E6572206D6F15
:1060500064650053657474696E6773207361766557
:106060006420746F20454550524F4D0A00526576AA
:1060700065727465642073657474696E67732066F5
:10608000726F6D20454550524F4D0A004C6F616450
:10609000656420666163746F7279206465666175FA
:1060A0006C74730A004B657920616E6420636861CB
:1060B0006E6E656C732072616E646F6D697A656473
:1060C0000A004F70656E4C52536E6720545820730F
:1060D00074617274696E672000206F6E20485720CB
:1060E0000050504D00525353490053444100534314
:1060F0004C00525844005458440041494E004C4210
:106100004545500053504B54524D00534255530097
:1061100053554D44004C4C494E440000342B340040
:106120003800382B340031320031322B3400313614
:106130000001000000C01200001A400AA1204EA574
:10614000001B1E27522C23308025000005400AA189
:10615000204EA50020244EA52C2330004B00000625
:10616000400AD0009D49007B289D492C233000E146
:10617000000005400A4501D7DC03B81E0EBF00230E
:106180002E48E801008A400A6001555502AD1E20E4
:10619000000023C88025000005400AA1204EA5006C
:1061A00020244EA52C233000020002000200020031
:1061B00002000200020002000200020002000200CF
:1061C00002000200020002FF610265026A026E0222
:1061D000720276027A027E0284028B02900295029B
:1061E0009B029B029B029B0235019C02A002A20221
:1061F000A602A902AE02350100070B0C1011150012
:10620000160A13223129000000005F2ECE2AEC2D41
:06621000262E062E4F2E83
:00000001FF
